S021000070726F6A656B745F77796B6C61645F365F6672656572746F732E73726563BB
S214080000F0A9002061010800E9010800E9010800DC
S214080010E9010800E9010800E901080000000000FD
S214080020000000000000000000000000B106080004
S214080030E90108000000000091080800D908080037
S214080040E9010800E9010800E9010800E9010800DB
S214080050E9010800E9010800E9010800E9010800CB
S214080060E9010800E901080000000000E9010800AD
S214080070E9010800E9010800E9010800000000009D
S21408008000000000E9010800E9010800E90108008D
S214080090E9010800E9010800E9010800E90108008B
S2140800A0E901080000000000E9010800E90108006D
S2140800B0E9010800E9010800E9010800E90108006B
S2140800C0E9010800E9010800E9010800E90108005B
S2140800D0E9010800E9010800E9010800E90108004B
S2140800E0E9010800E9010800E9010800E90108003B
S2140800F0E901080010B5054C237833B9044B13B151
S2140801000448AFF300800123237010BD3404002098
S21408011000000000282B08000C4B43B10C4810B513
S2140801200C49AFF300800C48036823B910BD0A4891
S214080130036833B97047094B002BF7D0BDE8104069
S2140801401847064B002BF5D0184700BF00000000E4
S214080150282B080038040020282B08000000000080
S21408016080B582B000AF174B7B60174B3B607A6850
S2140801703B689A420CD007E03B681A1D3A607A68DA
S214080180111D796012681A603B68104A9342F3D3CF
S2140801900F4B3B6004E03B681A1D3A6000221A6069
S2140801A03B680C4A9342F6D30B4B7B600B4A7B6842
S2140801B023F0604323F07F039360094B9847094B6D
S2140801C09847FEE7282B080000000020340400208B
S2140801D034040020ECA500200000080000ED00E034
S2140801E0D92708005505080080B400AFFEE70000D0
S2140801F080B584B000AF78600023FB607B6803F0AE
S2140802000703002B04D07B6823F0070308337B60C2
S214080210194B9847194B1B68002B05D1184B23F030
S21408022007031A46154B1A60164B1A687B68134460
S21408023049F6F772934213D8124B1A687B681A4429
S214080240104B1B689A420BD90C4B1A680D4B1B684F
S2140802501344FB600B4B1A687B681344094A136007
S214080260094B9847FB68002B01D1084B9847FB6859
S21408027018461037BD4680BD0517080054A4002050
S2140802805804002050A400202117080089040800FC
S21408029080B485B000AF78607B68002B09D04FF03B
S2140802A0A00383F31188BFF36F8FBFF34F8FFB60F4
S2140802B0FEE700BF1437BD4680BC704780B400AF69
S2140802C0044B1B68C3F51F43F8331846BD4680BC6D
S2140802D0704700BF50A4002080B483B000AF786099
S2140802E07B6803F108027B685A607B684FF0FF3230
S2140802F09A607B6803F108027B68DA607B6803F122
S21408030008027B681A617B6800221A6000BF0C37F7
S214080310BD4680BC704780B483B000AF78607B6809
S21408032000221A6100BF0C37BD4680BC704780B4F7
S21408033085B000AF786039607B685B68FB603B68B7
S214080340FA685A60FB689A683B689A60FB689B681C
S2140803503A685A60FB683A689A603B687A681A6135
S2140803607B681B685A1C7B681A6000BF1437BD463A
S21408037080BC704780B485B000AF786039603B6851
S2140803801B68BB60BB68B3F1FF3F03D17B681B6982
S214080390FB600CE07B680833FB6002E0FB685B6888
S2140803A0FB60FB685B681A68BB689A42F6D9FB680C
S2140803B05A683B685A603B685B683A689A603B686C
S2140803C0FA689A60FB683A685A603B687A681A6105
S2140803D07B681B685A1C7B681A6000BF1437BD46CA
S2140803E080BC704780B485B000AF78607B681B69B6
S2140803F0FB607B685B687A6892689A607B689B6833
S2140804007A6852685A60FB685A687B689A4203D1D1
S2140804107B689A68FB685A607B6800221A61FB68EA
S2140804201B685A1EFB681A60FB681B681846143758
S214080430BD4680BC7047000080B400AF044B1B6804
S2140804400133034A136000BFBD4680BC704700BF37
S21408045058A4002080B582B000AF064B98470346E4
S2140804607B60054B1B680133034A136000BF0837DF
S214080470BD4680BDBD02080060A4002080B483B0DD
S21408048000AF78603960FEE780B400AFFEE7000092
S21408049090B585B000AF78606423FB600C4B186895
S2140804A00023FA6879680B4CA047B860BB68012B34
S2140804B004D0094B1B680133074A1360074B4FF0FB
S2140804C080521A60BFF34F8FBFF36F8FE6E700BF07
S2140804D0C4A50020710B080064A4002004ED00E009
S2140804E080B584B000AF7860164B1B681846164B6C
S2140804F098470346032B04D0144B1B680133134A52
S2140805001360104B1B6807F1080100221846104BB1
S2140805109847F860FB68012B0ED17B7A002B05D133
S2140805200A4B1B680133094A1360DDE7074B1B6853
S2140805300133064A1360D7E7044B1B680133034AA6
S2140805401360D1E7C4A50020B910080064A40020F1
S214080550D10E080090B585B002AF00220221032014
S2140805601A4B984702461A4B1A60194B1B68002B01
S21408057020D00023019302230093164B4FF47A727F
S21408058015491648164CA0470023019302230093EA
S214080590144B4FF47A7214491048114CA0470023A4
S2140805A001930123009300234FF47A720F491048F1
S2140805B00B4CA0470F4B984778600F4B98470F4B4C
S2140805C01B6801330D4A1360F9E700BFB90A080033
S2140805D0C4A50020D02A0800D42A080091040800E0
S2140805E0C1130800D22A0800DC2A0800E42A0800FA
S2140805F0E1040800BD020800611608005CA400209B
S21408060080B485B000AFF860B9607A60FB68043BD8
S214080610FB60FB684FF080721A60FB68043BFB6067
S214080620BB6823F00102FB681A60FB68043BFB60AA
S214080630084AFB681A60FB68143BFB607A68FB682C
S2140806401A60FB68203BFB60FB6818461437BD46FB
S21408065080BC70475906080080B485B000AF0023F8
S2140806607B60104B1B68B3F1FF3F09D04FF0A00327
S21408067083F31188BFF36F8FBFF34F8FFB60FEE7DE
S2140806804FF0A00383F31188BFF36F8FBFF34F8F2C
S214080690BB6000BF7B68002BFCD000BF1437BD468C
S2140806A080BC704704000020000000000000000026
S2140806B0074B19680868B0E8F00F80F30988BFF39D
S2140806C06F8F4FF0000080F311884EF00D0E7047C4
S2140806D084A4002000BF00BF06480068006880F3B6
S2140806E0088862B661B6BFF34F8FBFF36F8F00DF1F
S2140806F000BF00BF08ED00E080B584B000AF314B06
S214080700FB60FB681B78DBB27B60FB68FF221A7015
S214080710FB681B78DBB2FB70FB78DBB223F05F0369
S214080720DAB2294B1A70294B07221A6009E0274BC0
S2140807301B68013B254A1360FB78DBB25B00DBB223
S214080740FB70FB78DBB203F08003802BEFD01F4BE7
S2140807501B68C3F10703042B09D04FF0A00383F3EB
S2140807601188BFF36F8FBFF34F8FBB60FEE7174B41
S2140807701B681B02154A1360144B1B6803F4E063DE
S214080780124A13607B68DAB2FB681A70104A104B7C
S2140807901B6843F4700313600D4A0D4B1B6843F047
S2140807A0704313600B4B98470B4B00221A600B4B99
S2140807B098470B4B98470B4B98470023184610371B
S2140807C0BD4680BD00E400E07CA4002080A4002094
S2140807D020ED00E01D09080004000020D9060800E6
S2140807E01D1A08005906080080B483B000AF4FF001
S2140807F0A00383F31188BFF36F8FBFF34F8F7B601F
S2140808000E4B1B6801330D4A13600C4B1B68012BFB
S2140808100ED10B4B1B68DBB2002B09D04FF0A003A0
S21408082083F31188BFF36F8FBFF34F8F3B60FEE7EC
S21408083000BF0C37BD4680BC704700BF04000020D0
S21408084004ED00E080B483B000AF104B1B68002BAB
S21408085009D14FF0A00383F31188BFF36F8FBFF35E
S2140808604F8F7B60FEE7094B1B68013B074A136006
S214080870064B1B68002B04D100233B603B6883F3C0
S214080880118800BF0C37BD4680BC704704000020A6
S214080890EFF30980BFF36F8F0D4B1A6820E9F00F4E
S2140808A010602DE908404FF0A00080F3118801F091
S2140808B0B5F84FF0000080F31188BDE808401968C5
S2140808C00868B0E8F00F80F30988BFF36F8F7047A9
S2140808D084A4002000BF00BF80B582B000AF4FF0F0
S2140808E0A00383F31188BFF36F8FBFF34F8F7B602E
S2140808F0084B98470346002B03D0074B4FF080520F
S2140809001A6000233B603B6883F3118800BF0837F2
S214080910BD4680BD8D18080004ED00E080B400AF29
S2140809200A4B00221A600A4B00221A60094A0A4B30
S2140809301B680A49A1FB03139B09013B1360034B81
S21408094007221A6000BFBD4680BC704710E000E072
S21408095018E000E014E000E000000020D34D62102C
S21408096080B485B000AFEFF30583FB60FB680F2B00
S21408097013D9154AFB6813441B78FB72134B1B7874
S214080980FA7A9A4209D24FF0A00383F31188BFF38C
S2140809906F8FBFF34F8F7B60FEE70D4B1B6803F42A
S2140809A0E0620C4B1B689A4209D94FF0A00383F308
S2140809B01188BFF36F8FBFF34F8F3B60FEE700BF12
S2140809C01437BD4680BC7047F0E300E07CA40020E6
S2140809D00CED00E080A4002080B584B000AF7860FD
S2140809E039607B68FB60FB68002B09D14FF0A003D9
S2140809F083F31188BFF36F8FBFF34F8FBB60FEE79B
S214080A00284B9847FB681A68FB68DB6BF968096C23
S214080A1001FB03F31A44FB689A60FB6800229A639A
S214080A20FB681A68FB685A60FB681A68FB68DB6B29
S214080A30013BF968096C01FB03F31A44FB68DA60AA
S214080A40FB68FF2283F84420FB68FF2283F84520D2
S214080A503B68002B14D1FB681B69002B1AD0FB6877
S214080A6010331846104B98470346002B12D00F4BEE
S214080A704FF080521A60BFF34F8FBFF36F8F09E0B5
S214080A80FB68103318460A4B9847FB682433184609
S214080A90074B9847074B9847012318461037BD461B
S214080AA080BD00BFE9070800CD1B080004ED00E084
S214080AB0D90208004508080090B58BB002AFF86068
S214080AC0B9601346FB71FB68002B09D14FF0A003F1
S214080AD083F31188BFF36F8FBFF34F8F3B61FEE739
S214080AE0FB68BA6802FB03F3FB61FB6948331846E8
S214080AF00C4B9847B861BB69002B0DD0BB697B616E
S214080B007B6948337B61FA79BB69009313467A6937
S214080B10B968F868044CA047BB6918462437BD4630
S214080B2090BD00BFF10108002D0B080080B584B009
S214080B3000AFF860B9607A60FB70BB68002B03D121
S214080B40BB69BA691A6002E0BB697A681A60BB6951
S214080B50FA68DA63BB69BA681A640121B869034B94
S214080B60984700BF1037BD4680BD00BFD9090800AA
S214080B7080B58EB000AFF860B9607A603B6000233D
S214080B807B63FB683B633B6B002B09D14FF0A003EC
S214080B9083F31188BFF36F8FBFF34F8FBB62FEE7F7
S214080BA0BB68002B03D13B6B1B6C002B01D10123C8
S214080BB000E00023002B09D14FF0A00383F311882F
S214080BC0BFF36F8FBFF34F8F7B62FEE73B68022B46
S214080BD003D13B6BDB6B012B01D1012300E0002323
S214080BE0002B09D14FF0A00383F31188BFF36F8F52
S214080BF0BFF34F8F3B62FEE7594B98470346002BDF
S214080C0002D17B68002B01D1012300E00023002BD2
S214080C1009D14FF0A00383F31188BFF36F8FBFF39A
S214080C204F8FFB61FEE74F4B98473B6B9A6B3B6BCE
S214080C30DB6B9A4202D33B68022B29D13A68B96823
S214080C40386B494B9847F8623B6B5B6A002B10D0B1
S214080C503B6B24331846454B98470346002B13D066
S214080C60434B4FF080521A60BFF34F8FBFF36F8F1E
S214080C700AE0FB6A002B07D03D4B4FF080521A6003
S214080C80BFF34F8FBFF36F8F3A4B9847012363E04C
S214080C907B68002B03D1374B984700235CE07B6BBF
S214080CA0002B06D107F114031846334B9847012347
S214080CB07B63304B9847314B98472A4B98473B6B9A
S214080CC093F844305BB2B3F1FF3F03D13B6B00228D
S214080CD083F844203B6B93F845305BB2B3F1FF3F93
S214080CE003D13B6B002283F84520224B98473A1DD8
S214080CF007F1140311461846214B98470346002B64
S214080D0024D1386B1F4B98470346002B18D03B6BF3
S214080D1010337A68114618461B4B9847386B1B4B9E
S214080D2098471B4B98470346002B7FF47CAF104B25
S214080D304FF080521A60BFF34F8FBFF36F8F72E782
S214080D40386B124B9847124B98476CE7386B0F4B2B
S214080D5098470F4B9847002318463837BD4680BD3E
S214080D60351F0800E9070800FD100800CD1B08001D
S214080D7004ED00E045080800991C0800051708005F
S214080D80C51C080011130800211B080029120800BA
S214080D902117080080B590B000AFF860B9607A6097
S214080DA03B60FB68BB63BB6B002B09D14FF0A0030D
S214080DB083F31188BFF36F8FBFF34F8FBB62FEE7D5
S214080DC0BB68002B03D1BB6B1B6C002B01D1012326
S214080DD000E00023002B09D14FF0A00383F311880D
S214080DE0BFF36F8FBFF34F8F7B62FEE73B68022B24
S214080DF003D1BB6BDB6B012B01D1012300E0002381
S214080E00002B09D14FF0A00383F31188BFF36F8F2F
S214080E10BFF34F8F3B62FEE72A4B9847EFF31182EA
S214080E204FF0A00383F31188BFF36F8FBFF34F8F84
S214080E30FA61BB61FB697B63BB6B9A6BBB6BDB6B55
S214080E409A4202D33B68022B2FD1BB6B93F84530EE
S214080E5087F83330BB6B9B6BFB623A68B968B86B34
S214080E60194B984797F93330B3F1FF3F12D1BB6B54
S214080E705B6A002B16D0BB6B24331846134B984777
S214080E800346002B0ED07B68002B0BD07B68012214
S214080E901A6007E097F833300133DBB25AB2BB6BFF
S214080EA083F845200123FB6301E00023FB637B6B8B
S214080EB07B617B6983F31188FB6B18464037BD4618
S214080EC080BD00BF61090800FD100800CD1B0800A2
S214080ED080B58CB000AFF860B9607A600023FB621A
S214080EE0FB68BB62BB6A002B09D14FF0A00383F3F3
S214080EF01188BFF36F8FBFF34F8F3B62FEE7BB6867
S214080F00002B03D1BB6A1B6C002B01D1012300E028
S214080F100023002B09D14FF0A00383F31188BFF3F9
S214080F206F8FBFF34F8FFB61FEE7564B984703461C
S214080F30002B02D17B68002B01D1012300E000239F
S214080F40002B09D14FF0A00383F31188BFF36F8FEE
S214080F50BFF34F8FBB61FEE74B4B9847BB6A9B6B53
S214080F607B627B6A002B1FD0B968B86A474B9847E4
S214080F707B6A5A1EBB6A9A63BB6A1B69002B0FD032
S214080F80BB6A10331846424B98470346002B07D0D7
S214080F90404B4FF080521A60BFF34F8FBFF36F8FEE
S214080FA03D4B9847012369E07B68002B03D13A4BF9
S214080FB09847002362E0FB6A002B06D107F110036E
S214080FC01846364B98470123FB62334B9847344BF9
S214080FD098472D4B9847BB6A93F844305BB2B3F1F9
S214080FE0FF3F03D1BB6A002283F84420BB6A93F80C
S214080FF045305BB2B3F1FF3F03D1BB6A002283F8EA
S2140810004520254B98473A1D07F110031146184608
S214081010244B98470346002B23D1B86A224B98479F
S2140810200346002B17D0BB6A24337A681146184645
S2140810301E4B9847B86A1E4B98471E4B9847034660
S214081040002B89D1134B4FF080521A60BFF34F8F95
S214081050BFF36F8F80E7B86A154B9847154B9847CC
S2140810607AE7B86A124B9847124B9847B86A0E4BFD
S21408107098470346002B3FF46FAF002318463037D7
S214081080BD4680BD351F0800E9070800D9110800CD
S214081090CD1B080004ED00E045080800991C080070
S2140810A005170800C51C0800DD120800211B0800EB
S2140810B0291208002117080080B584B000AF7860B0
S2140810C07B68002B09D14FF0A00383F31188BFF388
S2140810D06F8FBFF34F8FBB60FEE7064B98477B6862
S2140810E09B6BFB60044B9847FB6818461037BD4659
S2140810F080BD00BFE90708004508080080B586B02F
S21408110000AFF860B9607A6000237B61FB689B6B70
S2140811103B61FB681B6C002B0DD1FB681B68002B22
S2140811204DD1FB689B681846294B98477861FB6841
S21408113000229A6043E07B68002B19D1FB68586848
S214081140FB681B6C1A46B968224B9847FB685A68B6
S214081150FB681B6C1A44FB685A60FB685A68FB6895
S2140811609B689A422BD3FB681A68FB685A6026E08D
S214081170FB68D868FB681B6C1A46B968154B984715
S214081180FB68DA68FB681B6C5B421A44FB68DA602B
S214081190FB68DA68FB681B689A4207D2FB689A689D
S2140811A0FB681B6C5B421A44FB68DA607B68022BA0
S2140811B005D13B69002B02D03B69013B3B613B698B
S2140811C05A1CFB689A637B6918461837BD4680BD6B
S2140811D0711F08002928080080B582B000AF786023
S2140811E039607B681B6C002B18D07B68DA687B68D4
S2140811F01B6C1A447B68DA607B68DA687B689B68D5
S2140812009A4203D37B681A687B68DA607B68D96879
S2140812107B681B6C1A463868024B984700BF08372D
S214081220BD4680BD2928080080B584B000AF786028
S214081230264B98477B6893F84530FB7311E07B682C
S2140812405B6A002B12D07B6824331846204B9847DD
S2140812500346002B01D01F4B9847FB7B013BDBB2B4
S214081260FB7397F90F30002BE9DC00E000BF7B68C2
S214081270FF2283F84520184B9847144B98477B68FD
S21408128093F84430BB7311E07B681B69002B12D0BF
S2140812907B68103318460E4B98470346002B01D040
S2140812A00C4B9847BB7B013BDBB2BB7397F90E3000
S2140812B0002BE9DC00E000BF7B68FF2283F84420AF
S2140812C0054B984700BF1037BD4680BDE9070800A4
S2140812D0CD1B0800911D08004508080080B584B09D
S2140812E000AF7860084B98477B689B6B002B02D151
S2140812F00123FB6001E00023FB60044B9847FB6872
S21408130018461037BD4680BDE9070800450808009E
S21408131080B584B000AF7860094B98477B689A6BB5
S2140813207B68DB6B9A4202D10123FB6001E0002355
S214081330FB60044B9847FB6818461037BD4680BDCF
S214081340E90708004508080080B586B000AFF860D1
S214081350B9607A60FB687B61154B98477B6993F8A0
S21408136044305BB2B3F1FF3F03D17B69002283F8B8
S21408137044207B6993F845305BB2B3F1FF3F03D155
S2140813807B69002283F845200A4B98477B699B6B4C
S214081390002B06D17B6924337A68B9681846064B51
S2140813A098477869054B984700BF1837BD4680BDF3
S2140813B0E907080045080800711B080029120800FC
S2140813C090B58DB004AFF860B9603B601346FB80FB
S2140813D0FB889B0018461B4B984778617B69002B57
S2140813E00ED05020174B9847F861FB69002B03D0A6
S2140813F0FB697A691A6305E07869134B984701E038
S2140814000023FB61FB69002B13D0FA8800230393A3
S214081410FB6902937B6B01933B6B00933B68B9684F
S214081420F8680A4CA047F869094B98470123BB613E
S21408143002E04FF0FF33BB61BB6918462437BD4650
S21408144090BD00BFF101080091020800551408007D
S2140814507D15080080B588B000AFF860B9607A607E
S2140814603B603B6B186B7B689B001A46A521404B7C
S21408147098473B6B1A6B7B6803F18043013B9B00E4
S2140814801344BB61BB6923F00703BB61BB6903F068
S2140814900703002B09D04FF0A00383F31188BFF38E
S2140814A06F8FBFF34F8F7B61FEE7BB68002B1FD0A3
S2140814B00023FB6112E0BA68FB69134419783A6B9B
S2140814C0FB69134434330A461A70BA68FB69134436
S2140814D01B78002B06D0FB690133FB61FB69092BDF
S2140814E0E9D900E000BF3B6B002283F83D2003E00B
S2140814F03B6B002283F83420BB6A042B01D90423F3
S214081500BB623B6BBA6ADA623B6BBA6A1A643B6BBD
S21408151000225A643B6B04331846164B98473B6BBD
S21408152018331846134B98473B6B3A6B1A61BB6ADD
S214081530C3F105023B6B9A613B6B3A6B5A623B6B95
S21408154000229A643B6B002283F84C203A68F968BC
S214081550B869094B984702463B6B1A60FB6A002B32
S21408156002D0FB6A3A6B1A6000BF2037BD4680BDC2
S21408157015290800170308000106080080B582B080
S21408158000AF78602B4B98472B4B1B6801332A4AD1
S21408159013602A4B1B68002B09D1284A7B68136006
S2140815A0254B1B68012B10D1254B98470DE0254B82
S2140815B01B68002B09D1214B1B68DA6A7B68DB6A3B
S2140815C09A4202D81D4A7B6813601F4B1B6801337A
S2140815D01D4A13607B68DB6A01229A401B4B1B6816
S2140815E013431A4A13607B68DA6A13469B0013444F
S2140815F09B00174A1A447B68043319461046154B55
S2140816009847154B98470F4B1B68002B0ED00B4B73
S2140816101B68DA6A7B68DB6A9A4207D20F4B4FF080
S21408162080521A60BFF34F8FBFF36F8F00BF083723
S214081630BD4680BDE90708005CA5002084A40020FC
S214081640E51D080068A5002078A5002064A50020F0
S21408165088A400202F0308004508080004ED00E0D1
S21408166090B587B002AF1E4B01930023009300236A
S21408167082221C491C481D4CA047F860FB68012BB9
S21408168002D11B4B9847F860FB68012B15D14FF029
S214081690A00383F31188BFF36F8FBFF34F8FBB6030
S2140816A0144B4FF0FF321A60134B01221A60134B8B
S2140816B000221A60124B98470DE0FB68B3F1FF3F13
S2140816C009D14FF0A00383F31188BFF36F8FBFF3E0
S2140816D04F8F7B60FEE700BF1437BD4690BD00BF46
S2140816E080A50020F02A0800A91D0800C1130800DC
S2140816F0592108007CA5002068A5002060A50020C8
S214081700F906080080B400AF044B1B680133034A8F
S214081710136000BFBD4680BC704700BF84A500208C
S21408172080B584B000AF0023FB600023BB60414B4C
S2140817301B68002B09D14FF0A00383F31188BFF371
S2140817406F8FBFF34F8F3B60FEE73B4B9847394B95
S2140817501B68013B374A1360364B1B68002B61D168
S214081760364B1B68002B5DD02EE0354BDB68DB68FC
S214081770FB60FB6818331846324B9847FB680433FF
S2140817801846304B9847FB68DB6A01229A402E4B76
S2140817901B6813432C4A1360FB68DA6A13469B00DF
S2140817A013449B00294A1A44FB680433194610461A
S2140817B0274B9847FB68DA6A264B1B68DB6A9A420F
S2140817C002D3254B01221A601D4B1B68002BCCD177
S2140817D0FB68002B01D0214B9847214B1B687B6088
S2140817E07B68002B10D01F4B98470346002B02D06F
S2140817F0194B01221A607B68013B7B607B68002BD3
S214081800F1D1174B00221A60134B1B68002B09D026
S2140818100123BB60144B4FF080521A60BFF34F8F02
S214081820BFF36F8F114B9847BB6818461037BD46F5
S21408183080BD00BF84A50020E90708005CA500203D
S2140818401CA50020E503080064A5002088A4002045
S2140818502F03080084A4002070A50020F51E0800A9
S2140818606CA500208D18080004ED00E04508080067
S21408187080B483B000AF044B1B687B607B68184657
S2140818800C37BD4680BC704760A5002080B586B082
S21408189000AF00237B61524B1B68002B40F09380FF
S2140818A0504B1B6801333B614E4A3B6913603B69EA
S2140818B0002B1FD14C4B1B681B68002B09D04FF020
S2140818C0A00383F31188BFF36F8FBFF34F8F3B607E
S2140818D0FEE7454B1B68FB60444B1B68424A136097
S2140818E0424AFB681360424B1B680133404A136048
S2140818F0404B9847404B1B683A699A4248D33A4B44
S2140819001B681B68002B04D13B4B4FF0FF321A6054
S2140819103EE0354B1B68DB68DB68BB60BB685B6812
S2140819207B603A697B689A4203D2334A7B681360C5
S2140819302EE0BB6804331846304B9847BB689B6A52
S214081940002B04D0BB68183318462C4B9847BB6846
S214081950DB6A01229A402A4B1B681343284A136005
S214081960BB68DA6A13469B0013449B00254A1A4450
S214081970BB68043319461046234B9847BB68DA6A97
S214081980224B1B68DB6A9A42B9D301237B61B6E710
S2140819901E4B1B68DA6A1B4913469B0013449B00C0
S2140819A00B441B68012B01D901237B61184B1B686C
S2140819B0002B01D1174B9847174B1B68002B09D0F3
S2140819C001237B6106E0124B1B680133104A136043
S2140819D0104B98477B6918461837BD4680BD00BF30
S2140819E084A5002060A5002014A5002018A50020C6
S2140819F074A50020F51E08007CA50020E503080055
S214081A0064A5002088A400202F03080084A40020D2
S214081A106CA500205504080070A5002080B588B085
S214081A2000AF394B1B68002B03D0384B01221A60D5
S214081A3065E0364B00221A60354B1B681B6BFB6152
S214081A404FF0A533BB61FB691A68BB699A4211D18E
S214081A50FB6904331A68BB699A420BD1FB690833E1
S214081A601A68BB699A4205D1FB690C331A68BB69C8
S214081A709A4208D0264B1A68254B1B6834331946F9
S214081A801046244B9847244B1B68FB60FB68B3FA48
S214081A9083F3FB72FB7AC3F11F037B611F497A69E4
S214081AA013469B0013449B000B441B68002B09D16C
S214081AB04FF0A00383F31188BFF36F8FBFF34F8FE8
S214081AC07B60FEE77A6913469B0013449B00134A23
S214081AD013443B613B695B685A683B695A603B69DB
S214081AE05A683B6908339A4204D13B695B685A686E
S214081AF03B695A603B695B68DB68054A136000BF50
S214081B002037BD4680BD00BF84A5002070A50020F4
S214081B1084A400207D04080064A5002088A4002072
S214081B2080B584B000AF786039607B68002B09D137
S214081B304FF0A00383F31188BFF36F8FBFF34F8F67
S214081B40FB60FEE7074B1B68183319467868064B98
S214081B50984701213868054B984700BF1037BD469F
S214081B6080BD00BF84A400207503080081200800FB
S214081B7080B586B000AFF860B9607A60FB68002B65
S214081B8009D14FF0A00383F31188BFF36F8FBFF31B
S214081B904F8F7B61FEE70A4B1B6818331946F868B7
S214081BA0084B98477B68002B02D04FF0FF33BB608A
S214081BB07968B868044B984700BF1837BD4680BD9B
S214081BC084A400202F0308008120080080B586B072
S214081BD000AF78607B68DB68DB683B613B69002B9D
S214081BE009D14FF0A00383F31188BFF36F8FBFF3BB
S214081BF04F8FFB60FEE73B69183318461E4B984725
S214081C001E4B1B68002B1CD13B69043318461A4B25
S214081C1098473B69DB6A01229A40194B1B681343B5
S214081C20174A13603B69DA6A13469B0013449B0005
S214081C30144A1A443B69043319461046124B98470F
S214081C4005E03B691833194610480F4B98473B691F
S214081C50DA6A0F4B1B68DB6A9A4205D901237B6157
S214081C600C4B01221A6001E000237B617B69184651
S214081C701837BD4680BD00BFE503080084A50020D0
S214081C8064A5002088A400202F0308001CA50020B7
S214081C9084A4002070A5002080B483B000AF7860CC
S214081CA0064B1A687B681A60054B1A687B685A6088
S214081CB000BF0C37BD4680BC704700BF74A5002027
S214081CC060A5002080B588B000AF786039607B6872
S214081CD0002B09D14FF0A00383F31188BFF36F8F51
S214081CE0BFF34F8F3B61FEE73B68002B09D14FF0EF
S214081CF0A00383F31188BFF36F8FBFF34F8FFB608A
S214081D00FEE71E4B98471E4B1B68BB617B685B68EB
S214081D10BA69D31A7B613B681B68B3F1FF3F02D1EF
S214081D200023FB6123E07B681A68164B1B689A42FF
S214081D3007D07B685A68BB699A4202D80123FB61C0
S214081D4015E03B681A687B699A420BD93B681A68A3
S214081D507B69D21A3B681A6078680B4B9847002351
S214081D60FB6104E03B6800221A600123FB61074B15
S214081D709847FB6918462037BD4680BDE907080026
S214081D8060A5002074A50020991C080045080800D6
S214081D9080B400AF034B01221A6000BFBD4680BC6A
S214081DA0704700BF70A5002080B582B000AF78608D
S214081DB0084B9847084B1B68012B07D9074B4FF071
S214081DC080521A60BFF34F8FBFF36F8F044B98474C
S214081DD0EEE700BF691E080088A4002004ED00E0B6
S214081DE03904080080B582B000AF00237B600CE0A1
S214081DF07A6813469B0013449B00124A13441846FD
S214081E00114B98477B6801337B607B68042BEFD9BE
S214081E100E480D4B98470E480B4B98470D480A4BF3
S214081E2098470D48084B98470C48074B98470C4B63
S214081E30064A1A600B4B064A1A6000BF0837BD46AA
S214081E4080BD00BF88A40020D9020800ECA40020AA
S214081E5000A500201CA5002030A5002048A50020CD
S214081E6014A5002018A5002080B582B000AF19E0A0
S214081E70104B9847104BDB68DB687B607B68043345
S214081E8018460E4B98470E4B1B68013B0C4A1360CE
S214081E900C4B1B68013B0B4A13600B4B9847786842
S214081EA00A4B9847074B1B68002BE1D100BF083741
S214081EB0BD4680BDE907080030A50020E5030800F8
S214081EC05CA5002044A5002045080800D11E08008F
S214081ED080B582B000AF78607B681B6B1846044BF1
S214081EE098477868024B984700BF0837BD4680BDBC
S214081EF09102080080B483B000AF0C4B1B681B68C7
S214081F00002B04D10A4B4FF0FF321A6008E0074B4B
S214081F101B68DB68DB687B607B685B68044A136069
S214081F2000BF0C37BD4680BC704700BF14A5002014
S214081F307CA5002080B483B000AF0B4B1B68002B39
S214081F4002D101237B6008E0084B1B68002B02D1F6
S214081F5002237B6001E000237B607B6818460C3711
S214081F60BD4680BC704700BF68A5002084A5002039
S214081F7080B586B000AF78607B683B6100237B61E4
S214081F807B68002B6CD0394B1B683A699A4209D09B
S214081F904FF0A00383F31188BFF36F8FBFF34F8F03
S214081FA0FB60FEE73B695B6C002B09D14FF0A00392
S214081FB083F31188BFF36F8FBFF34F8FBB60FEE7C5
S214081FC03B695B6C5A1E3B695A643B69DA6A3B6933
S214081FD01B6C9A4244D03B695B6C002B40D13B6932
S214081FE004331846224B98470346002B15D13B6905
S214081FF0DA6A204913469B0013449B000B441B686F
S214082000002B0AD13B69DB6A012202FA03F3DA43A2
S214082010194B1B681340184A13603B691A6C3B69D6
S214082020DA623B69DB6AC3F105023B699A613B6980
S214082030DB6A01229A40104B1B6813430E4A136052
S2140820403B69DA6A13469B0013449B00094A1A4404
S2140820503B69043319461046084B984701237B61B1
S2140820607B6918461837BD4680BD00BF84A400208B
S214082070E503080088A4002064A500202F030800B4
S21408208080B584B000AF78603960294B1B68FB6068
S214082090284B1B6804331846274B98470346002BE3
S2140820A00BD1244B1B68DB6A012202FA03F3DA43DE
S2140820B0224B1B681340214A13607B68B3F1FF3F2D
S2140820C00AD13B68002B07D01A4B1B680433194605
S2140820D01B481C4B984726E0FA687B681344BB608D
S2140820E0144B1B68BA685A60BA68FB689A4209D2E9
S2140820F0154B1A680F4B1B68043319461046134BCA
S214082100984710E0124B1A680A4B1B6804331946A6
S21408211010460E4B98470F4B1B68BA689A4202D275
S2140821200C4ABB68136000BF1037BD4680BD00BFB1
S21408213060A5002084A40020E503080064A500200C
S21408214048A500202F03080018A5002075030800DE
S21408215014A500207CA5002090B585B002AF00230A
S2140821607B60124B9847124B1B68002B0BD0114B09
S21408217001930223009300234FF482720E490F48FE
S2140821800F4CA04778607B68002B09D14FF0A0035E
S21408219083F31188BFF36F8FBFF34F8F3B60FEE763
S2140821A07B6818460C37BD4690BD00BF75270800EB
S2140821B0B8A50020BCA50020F82A08000D230800B2
S2140821C0C113080090B58BB000AFF860B9607A60AC
S2140821D03B6000237B62FB68002B09D14FF0A0030D
S2140821E083F31188BFF36F8FBFF34F8F3B62FEE711
S2140821F0194B1B68002B2AD0BB687B617B68BB61C8
S214082200FB68FB61BB68052B18DC144B9847034634
S214082210022B09D1104B186807F114010023BA6B7A
S2140822200F4CA047786212E00B4B186807F11401B0
S214082230002300220A4CA047786208E0064B18687C
S21408224007F1140100233A68064CA04778627B6AB7
S21408225018462C37BD4690BDB8A50020351F080087
S214082260710B0800950D080090B589B002AF78602C
S2140822703960224B1B68DB68DB687B617B6904334B
S21408228018461F4B98477B6993F8243003F00403DD
S214082290002B21D07B699A697B68D1187B683A68DD
S2140822A07869184CA0470346002B1ED000230093DD
S2140822B000237A6800217869134CA04738613B6987
S2140822C0002B12D14FF0A00383F31188BFF36F8F52
S2140822D0BFF34F8FFB60FEE77B6993F8243023F04B
S2140822E00103DAB27B6983F824207B691B6A786964
S2140822F0984700BF1C37BD4690BD00BFB0A500205C
S214082300E503080079240800C521080080B584B0D4
S21408231000AF786007F108031846054B9847F86041
S214082320BB681946F868034B9847034B9847F1E78C
S214082330ED2308003D2308000125080080B584B079
S21408234000AF78603960214B984707F108031846B4
S2140823501F4B9847F860BB68002B30D13B68002BB2
S2140823600AD17A68FB689A4206D81A4B9847F968E1
S2140823707868194B984724E03B68002B08D0174B21
S2140823801B681B68002B01D1012300E000233B607B
S214082390134B18687A68FB68D31A3A681946114BC3
S2140823A098470C4B98470346002B0AD10E4B4FF024
S2140823B080521A60BFF34F8FBFF36F8F01E0054B53
S2140823C0984700BF1037BD4680BD00BF05170800F8
S2140823D0312408002117080069220800B4A5002047
S2140823E0B8A500204913080004ED00E080B485B0C5
S2140823F000AF78600D4B1B681B68002B01D10122CB
S21408240000E000227B681A607B681B68002B05D1F9
S214082410064B1B68DB681B68FB6001E00023FB605B
S214082420FB6818461437BD4680BC7047B0A5002028
S21408243080B584B000AF78600C4B9847F8600C4BBA
S2140824401B68FA689A4205D20A4B98477B680122AD
S2140824501A6002E07B6800221A60054AFB6813606F
S214082460FB6818461037BD4680BD00BF71180800C7
S214082470C0A50020A126080080B586B000AFF86089
S214082480B9607A603B6000237B61FB68BA685A6073
S214082490FB68FA681A61BA687B689A4212D87A6842
S2140824A03B68D21AFB689B699A4202D301237B6178
S2140824B01BE0104B1A68FB680433194610460E4B8F
S2140824C0984712E07A683B689A4206D2BA683B6830
S2140824D09A4202D301237B6107E0084B1A68FB681F
S2140824E0043319461046044B98477B691846183734
S2140824F0BD4680BDB4A5002075030800B0A5002021
S21408250090B58DB002AFACE0BB68002BC0F2A980D6
S2140825103B697B627B6A5B69002B04D07B6A043369
S2140825201846584B98473B1D1846574B98473862ED
S214082530BB68092B00F2948001A252F823F000BF72
S214082540692508006925080069250800DB250800B4
S214082550EF250800372608006925080069250800C1
S214082560DB250800EF2508007B6A93F8243043F043
S2140825700103DAB27B6A83F82420FA687B6A9B69CF
S214082580D118FB683A6A786A404CA0470346002B85
S21408259067D07B6A1B6A786A98477B6A93F8243008
S2140825A003F00403002B5CD0FA687B6A9B691A4424
S2140825B00023009300230021786A354CA047F86171
S2140825C0FB69002B4DD14FF0A00383F31188BFF3AE
S2140825D06F8FBFF34F8FBB61FEE77B6A93F824309B
S2140825E023F00103DAB27B6A83F8242039E07B6A99
S2140825F093F8243043F00103DAB27B6A83F8242088
S214082600FA687B6A9A617B6A9B69002B09D14FF04E
S214082610A00383F31188BFF36F8FBFF34F8F7B61DF
S214082620FEE77B6A9A693B6AD1183B6A3A6A786A17
S214082630164CA04715E07B6A93F8243003F0020393
S214082640002B03D1786A134B98470AE07B6A93F805
S214082650243023F00103DAB27B6A83F8242000E0F2
S21408266000BF0D4B1B6807F10801002218460B4BEC
S21408267098470346002B7FF447AF00BF2C37BD466C
S21408268090BD00BFE503080031240800792408003F
S214082690C521080091020800B8A50020D10E080040
S2140826A090B589B002AF47E02D4B1B68DB681B6806
S2140826B07B612B4B1B68DB68DB683B613B6904333B
S2140826C01846284B98473B691B6A386998473B6900
S2140826D093F8243003F00403002B2DD03B699A6945
S2140826E07B691344FB60FA687B699A420ED93B699A
S2140826F0FA685A603B693A691A61194B1A683B6965
S214082700043319461046184B984715E000230093E3
S21408271000237A6900213869144CA047B860BB6862
S214082720002B09D14FF0A00383F31188BFF36F8FF6
S214082730BFF34F8F3B60FEE7094B1B681B68002BF7
S214082740B2D1074B1B687B60094B1B68044A1360B1
S214082750074A7B68136000BF1C37BD4690BD00BFA4
S214082760B0A50020E503080075030800C521080089
S214082770B4A5002080B500AF0E4B98470E4B1B68DB
S214082780002B13D10D480E4B98470E480C4B984714
S2140827900D4B0A4A1A600D4B0A4A1A6000220C2191
S2140827A005200B4B98470246034B1A60094B98477F
S2140827B000BF80BDE9070800B8A5002088A500204E
S2140827C0D90208009CA50020B0A50020B4A50020CA
S2140827D0B90A08004508080070B50F4E0F4D761B5D
S2140827E0B61018BF002405D0013455F8043B9847A6
S2140827F0A642F9D10A4E0B4D00F084F9761BB610A6
S21408280018BF002406D0013455F8043B9847A64262
S214082810F9D170BD70BD00BF102B0800102B080042
S214082820182B0800102B0800844641EA000313F012
S214082830030349D1403A23D30B6803604B684360CF
S2140828408B688360CB68C3600B6903614B6943611F
S2140828508B698361CB69C3610B6A03624B6A436207
S2140828608B6A8362CB6AC3620B6B03634B6B4363EF
S2140828708B6B8363CB6BC36340304031403ADBD20B
S21408288030320BD30B6803604B6843608B688360F9
S214082890CB68C36010301031103AF3D20C3205D32F
S2140828A051F8043B40F8043B043AF9D2043208D005
S2140828B0D2071CBF11F8013B00F8013B01D30B8877
S2140828C003806046704700BF082A13D38B07B1D031
S2140828D010F00303AED0C3F10403D21ADB071CBF03
S2140828E011F8013B00F8013BA4D331F8023B20F86D
S2140828F0023B9FE7043AD9D3013A11F8013B00F8A6
S214082900013BF9D20B7803704B7843708B78837051
S2140829106046704770B4860746D0541E002A41D0D9
S214082920CAB2034602E014F1FF343BD303F8012B86
S2140829309D07F8D1032C2ED9CDB245EA05250F2CD4
S21408294045EA054519D9264603F11002103E0F2E12
S21408295042F8105C42F80C5C42F8085C42F8045CEA
S21408296002F11002F2D8A4F1100222F00F0204F0CD
S2140829700F041032032C13440DD91E462246043A7F
S214082980032A46F8045BFAD8221F22F00302043210
S214082990134404F003042CB1C9B21C4403F8011B09
S2140829A09C42FBD170BC704714460346C2E700BF82
S2140829B0024B13B1024800F005B87047000000004B
S2140829C0D1290800002301461A46184600F01EB80A
S2140829D038B50A4C0A4D641BA4100AD004F180438B
S2140829E0013B05EB8305013C55F804399847002C54
S2140829F0F9D1BDE8384000F08FB800BF282B080092
S214082A00242B0800704700BF704700BF2DE9F84325
S214082A102C4D0646286898460F469146FFF7F2FF63
S214082A20294B1C68D4F84831002B3ED05A681F2A18
S214082A301CDC02F1010E76B1012103EB8204C4F816
S214082A408890D3F8880191400843022EC3F888017D
S214082A50C4F8088123D00232C3F804E0286843F893
S214082A602270FFF7D1FF0020BDE8F883174B0BB3A1
S214082A704FF4C870AFF300800346D8B10020D4F8EE
S214082A8048114FF0010E586019600246C4F84831E4
S214082A90C3F88801C3F88C01002EDCD0CCE7D3F845
S214082AA08C010143C3F88C11D5E704F5A673C4F866
S214082AB04831BBE72868FFF7A7FF4FF0FF30BDE8AF
S214082AC0F88300BF30040020002B08000000000038
S214082AD06400C80153656E646572310053656E64A0
S214082AE0657232005265636569766572000000009B
S214082AF049444C4500000000546D7220537663002C
S214082B0008000020F8B500BFF8BC08BC9E46704711
S214082B10B129080019010800F8B500BFF8BC08BCC0
S20C082B209E467047F500080008
S214082B2800093D00AAAAAAAA00000000F40200208C
S214082B385C030020C403002000000000000000001A
S214082B480000000000000000000000000000000070
S214082B580000000000000000000000000000000060
S214082B680000000000000000000000000000000050
S214082B780000000000000000000000000000000040
S214082B880000000000000000000000000000000030
S214082B980000000000000000000000000000000020
S214082BA80000000000000000000000000000000010
S214082BB80000000000000000000000000000000000
S214082BC800000000000000000000000000000000F0
S214082BD801000000000000000E33CDAB34126DE68D
S214082BE8ECDE05000B0000000000000000000000F6
S214082BF800000000000000000000000000000000C0
S214082C0800000000000000000000000000000000AF
S214082C18000000000000000000000000000000009F
S214082C28000000000000000000000000000000008F
S208082F58C8A50020DB
S804080000F3
